:020000040000FA
:100000002500870C0200380C2E000600000C26008C
:10001000010C28003F0C2C006B00C80C810003076A
:100020000D0A610040094D02360E43066B000C02BA
:100030008D01090E36004D02360E160143060D0ADB
:100040000C020D01360F360E4307280A6B002C0AEE
:100050000C0C8B000307AB02030C8B000307000C96
:100060002800020CE8010D022C004F09100C24009E
:10007000050C370000028609A402F7023A0A0D0AAD
:10008000460406022D002D032D032D03070C6D01E0
:100090004605380C46012D01000C26000008870C8F
:1000A00030007100720073007400090C4D014307A9
:1000B0005B0A30045F0A0D0710046D075004030447
:1000C000080329002A000306AA02120C4D01430668
:1000D000750A09022D06700AF1010A02F301750A78
:1000E0008D06750AB1000A02B300240C4D014306C7
:1000F00000080802AD06800AF2010A02F4010008B5
:100100004D060008B2000A02B40000082700080CDF
:1001100035002605A2099C090706900A2605910AC2
:100120002604920A930A9C092703F5028C0A2604E6
:100130009C09A2099B0A0008CF0C2F000000EF02C7
:100140009E0A0008000000084208590820084A08D2
:0A0150004A0831084F0844084D0822
:021FFE00EA0FE8
:00000001FF
